:03000000023C9827
:0C3C980078FFE4F6D8FD75816F023CDF78
:1013FB000A53746172743A20004950436F6E6E65E4
:10140B0063745245510A004950436F6E6E656374A5
:10141B00003E432C562C43432CC0E4E0EFF2E5F0A6
:10142B0020D1E8EDEAEEEC49500A003E432C4D4149
:10143B00432C25303262583A25303262583A2530E7
:10144B003262583A25303262583A25303262583A75
:10145B0025303262582C4D414320E0E4F0E5F10A8F
:10146B00003E432C5645522C20332E3120EEF220D9
:10147B0025732025732CC2E5F0F1E8FF204950209D
:10148B00ECEEE4F3EBFF0A004E6F762030362032A1
:10149B003030370031303A31373A3237003E432C57
:1014AB004C442C50524F473A202020202020202003
:1014BB002020202020202020202020202020202021
:1014CB002020202020202020202020202020202011
:1014DB002020202020202020202020202020202001
:1014EB00202020202020202020202020202CC4E081
:1014FB00F2E020EFF0EEF8E8E2EAE828F4E0E9EBBE
:10150B00290A003E2A2C312CCEF1EDEEE2EDFBE563
:10151B0020EFE0F0E0ECE5F2F0FB20F1E5F2E5E2A4
:10152B00EEE3EE20E8EDF2E5F0F4E5E9F1E00A0098
:10153B003E412C4130312C2562752E2562752E25AE
:10154B0062752E2562752C495020E0E4F0E5F12000
:10155B00E0E4E0EFF2E5F0E00A003E412C413032EE
:10156B002C2562752E2562752E2562752E256275CA
:10157B002C495020E0E4F0E5F120EEF1ED2E20F1C6
:10158B00E5F0E2E5F0E00A003E412C4130332C253A
:10159B0062752E2562752E2562752E2562752C4976
:1015AB005020E0E4F0E5F120F0E5E72E20F1E5F046
:1015BB00E2E5F0E00A003E412C4130342C25627507
:1015CB002E2562752E2562752E2562752CCCE0F1C9
:1015DB00EAE020F1E5F2E80A003E412C4130352CDF
:1015EB002562752E2562752E2562752E2562752C4A
:1015FB00D8EBFEE70A003E532C4130362C256275A2
:10160B002CC2F0E5ECFF20EEE6E8E42E20EAE2E85F
:10161B00F2E0EDF6E8E820282A3130ECF1290A0057
:10162B003E2A2C312CC4EEEF2E20EFE0F0E0ECE55F
:10163B00F2F0FB20F1E5F2E5E2EEE3EE20E8EDF26D
:10164B00E5F0F4E5E9F1E00A003E422C5330312C91
:10165B002562752CC6E4E0F2FC20E7E0EFF0EEF13A
:10166B00E020F1EEE5E4E8EDE5EDE8FF20EEF22019
:10167B00F1E5F0E2E5F0E00A003E422C5330322C6B
:10168B002562752CCEE1ECE5ED20F120F1E5F0E2E1
:10169B00E5F0EEEC20E1E5E720EAE2E8F2E0EDF63A
:1016AB00E8E90A003E422C5330332C2562752CCFCF
:1016BB00E5F0E5E7E0EFF3F1EA20EFF0E820EFEEFD
:1016CB00F2E5F0E520F1E2FFE7E820F120F1E5F0AB
:1016DB00E2E5F0EEEC0A003E422C5330342C25624E
:1016EB00752CCDE5F220EFE5F0E5E4E0F7E820E43A
:1016FB00E8E0E3EDEEF1F2E8EAE820E220F1E5F0D4
:10170B00E2E5F00A003E422C5330352C2562752C55
:10171B00CAE0EDE0EB20F8E8F0EEEAEEE2E5F8E007
:10172B00F2E5EBFCEDEEE3EE20EEE1ECE5EDE00AAD
:10173B00003E532C5330362C253032625825303234
:10174B006258253032625825303262582530326269
:10175B005825303262582C4D414320E0E4F0E5F13E
:10176B0020F8E8F0EEEAEEE2E5F8E0F2E5EBFCED6E
:10177B00EEE3EE20EEE1ECE5EDE00A003E454E44F3
:10178B000A0044756D705820202020203030203006
:10179B003120303220303320303420303520303679
:1017AB002030372030382030392030412030422053
:1017BB0030432030442030452030460A003A200088
:1017CB000A0044756D7044202020202030302030DA
:1017DB003120303220303320303420303520303639
:1017EB002030372030382030392030412030422013
:1017FB0030432030442030452030460A0045727279
:10180B00206B657900526420656570726F6D0A00FC
:10181B005264204D454D0A00526420436F64650AA3
:10182B000044656275674950204F4E0A004465625B
:10183B0075674950204F46460A00446562756755E7
:10184B00736572204F6E0A00446562756755736548
:10185B0072204F46460A0044656275674D736720D8
:10186B004F6E0A0044656275674D7367204F46469D
:10187B000A00436F6E666967206C6F636B210A0009
:10188B00577220656570726F6D0A00205361766523
:10189B0020656570726F6D210A00457272204D4193
:1018AB004321004C6F61643E3E002A003C413031C5
:1018BB003D003C4130323D003C4130333D003C412A
:1018CB0030343D003C4130353D003C4130363D002D
:1018DB004E4F4950004C494E4B434F4E54520054BF
:1018EB0052415353004652004E4F4C494E4B004908
:1018FB004E49004E4F4449414700003C21003C53A8
:10190B0030313D003C5330323D003C5330333D00D1
:10191B003C5330343D003C5330353D003C53303666
:10192B003D00FF18DBFF18E0FF18EAFF18F0FF1867
:0A193B00F3FF18FAFF18FEFF19056C
:06466D00010B0001090031
:10462C00C2AFC28E438910758BFF758DB7D2ABD2DA
:04463C008ED2AF2249
:03001B00023B6E37
:103B6E00C0E0C083C082C0D0C2AFC28E758BFF755D
:103B7E008DB720060675A61E75A6E10509D202E5CB
:103B8E000B6002050BE50AD394014002150A050EDF
:103B9E00E50E540F7050D20DE50E543F701AD20040
:103BAE00907B01E0601204F0E0D394B4400A908060
:103BBE00007480F0C2AF80FE907AFCE0600204F0E8
:103BCE00907578E0600214F0907B02E0D39401408F
:103BDE0003E014F0300502050CE50DD394644004A7
:103BEE00D2068002050DE508D3940140021508D2D5
:0C3BFE008ED2AFD0D0D082D083D0E03285
:10088100C291C290D2B5C20A7D027C007F07124597
:10089100C08F25E525646060097D017F6012457880
:1008A100D20AE4FDFC7F0B1245C08F25E52530E619
:1008B100097D04E4FF12459CD20A7D017C007F077B
:1008C1001245C08F25E5257008FD7FFF124578D2BE
:1008D1000A300A03126000C2AFC288C2A8C2AA7558
:1008E1008900123F2D9077B5E0B4FA09A3E064CEF8
:1008F1007003020981E4F52574AD2525F582E43400
:1009010077F583E4F00525E525B443EC9077B574DC
:10091100FAF0A374CEF0A374CCF09077BB740AF014
:10092100E4A3F0A304F0A3F09077C07403F0A374E0
:10093100CCF09077B174FFF0A3F0A3F0E4A3F090B2
:1009410077CC7405F0E4F525E5252401FFE433FEB9
:1009510074AD2525F582E43477F583E0FD12461365
:100961000525E525C3944340DFE4F5A775A61E756B
:10097100A6E1907FF0F0A3F09080007480F080FEFB
:10098100D2AF9077C07403F0A374CCF0E49077BF3A
:10099100F01235E4EF600312271AC2B512290DC215
:1009A100061243019077CCE0C3940350037403F023
:1009B100D20AC20CC20BD293200A077E137FFB120C
:1009C10036CAE49079ECF012462CC2AFA37408F059
:1009D10090772B7424F0E4A3F09077B5E090772D15
:1009E100F09077B6E090772EF09077B7E090772F80
:1009F100F09077B8E0907730F09077B9E090773168
:100A0100F09077BAE0907732F0750A01E49079EED0
:100A1100F0C207C208D2AF75A70775A61E75A6E179
:100A2100124551200A19AF257E007D031237ABE430
:100A3100FF123A237E777FECE4FB7D01123885902B
:100A41007B01E060037401F0E4907578F0A37455C4
:100A5100F0A37481F0E4F50CE4F50D907578E07085
:100A610003121F68907B02E0B401119080007410A2
:100A7100F0E4907B02F0D20AD20BD20C908008E015
:100A8100F52530E405D2077410F0E52530E508D2EC
:100A9100099080087420F0E52530E608D20890809E
:100AA100087440F0E50CD394034023908002E4F0F5
:100AB100908001F0908000F0E50CD39406400FE4A3
:100AC100F50CC2039079EEF0750A01124301908092
:100AD100A0E070031240269080B8E070031240A09D
:100AE1009080D0E0700312417F908000E07013305D
:100AF10007101234E09077A8EFF0D394004003126E
:100B01000026908002E07006908000E06005D2052A
:100B1100020A59C205E4F50C907578E06003020AF7
:100B21005930091212311D9077A8EFF0D39400408B
:100B310005E0FF124640200803020CB8122E409037
:100B410077A8EFF07003020A599077ECE054BF24C4
:100B51007F7003020C1B147003020BF32402600369
:100B6100020C4E200A077E147F041236CA300E7919
:100B71002003769077C4E070069077C8E0605B90C0
:100B81007AF8E0FF9077C4E0B50724907AF9E0FEA7
:100B91009077C5E0B50618907AFAE0FE9077C6E046
:100BA100B5060C907AFBE0FE9077C7E06E602B9063
:100BB10077C8E06F7033907AF9E0FF9077C9E0B5BC
:100BC1000727907AFAE0FF9077CAE0B5071B907A81
:100BD100FBE0FF9077CBE0B5070F9079EE7401F061
:100BE100120021750A01020CB8907AF874FFF00224
:100BF1000CB8907B01E060037401F0907AF0E0FFA3
:100C01009077EEE06F6003020CB8907AF0E004F0A8
:100C1100E4F50A9079ECF0020CB8300303020CB849
:100C21009077BBE07003020A59124674D203E4F5CF
:100C31000A9079ECF0907AFC04F0E4907AEFF0A35A
:100C4100F0200A737E147F121236CA806A907B01EB
:100C5100E060037401F03003529077ECE020E74B41
:100C61009077EEE0FF907AEFE0FE6F600D907AF7FB
:100C7100E07007EE146F703F8013907AEFE004F09C
:100C81009077A8E0FFD3940440031243E890747472
:100C91007482F0A37401F09077EEE0907476F07EA8
:100CA100747F747D03123FAB020A59300E09200391
:100CB10006907AF874FFF0200303020D6DE50A70C7
:100CC1006B124499EF60207E787FEC9078EDE02400
:100CD10004FD123FAB907AF7E06003020A59907766
:100CE100CCE0F50A020A59907AFCE0D3943C403CEE
:100CF100907AF7E07036907AFC04F090772AE070F1
:100D01002B12465AE49078ECF0A37412F0907AF02A
:100D1100E09078EEF0A374FDF090757B63A20190F2
:100D210078F063A2017F12122BC5809B12464FEF10
:100D310060159074747483F0E4A3F07E747F747D05
:100D410002123FAB020A59E50A64016003020A5923
:100D51009079ECE004F0E0C394055003020CC8C2A2
:100D610003E49079EEF0120021020A59E50A6401C8
:100D71006003020A599079EEE014604024FE603C61
:100D8100147003020E5524046003020A59E4F50CA1
:100D9100200E139079EE7404F09079ECE05401F098
:100DA100750A01020A59E49079EEF09079EC04F0A9
:100DB100750AC8907AF874FFF0020A59907AF8E03F
:100DC1007003020E449078EC7480F09078EE740118
:100DD100F0E4A3F0A304F0A37430F0A3747BF0E477
:100DE100F52574F32525F582E43478F583747DF0D7
:100DF10074F42525F582E43478F583E4F0E52524BF
:100E0100079078EDF07C7A7DF89077C0E0FAA3E066
:100E1100FB7F02123DA97E787FECE5252409FD12B6
:100E21003FAB907AF7E0601B124674D203E4F50AF7
:100E31009079ECF0907AFC04F0E4907AEFF0A3F072
:100E4100020A599079EE7404F09077CCE02432F5DF
:100E51000A020A599080027410F0750A039079EC25
:100E6100E06401FFF09079EE7401F0EF7019907772
:100E7100C8E06013FCA3E0FDA3E0FEA3E0FF907ACD
:100E8100F8122376020A599077C4E0FCA3E0FDA38F
:100E9100E0FEA3E0FF907AF8122376020A5980FE61
:010EA100222E
:100026009077EDE0B444047F0180027F009077EC86
:10003600E0B447047E0180027E00EE5F604A90775E
:10004600B5E09077EEF09077B6E09077EFF09077A6
:10005600B7E09077F0F09077B8E09077F1F090778E
:10006600B9E09077F2F09077BAE09077F3F0907776
:10007600ED7452F090772463A2019080A863A201E8
:100086007F06122BC50208779077A8E0C394085024
:10009600030208809077B5E0FF9077EEE06F60038B
:1000A6000208809077B6E0FF9077EFE06F6003027A
:1000B60008809077B7E0FF9077F0E06F6003020862
:1000C600809077B8E0FF9077F1E06F6003020880D8
:1000D6009077B9E0FF9077F2E06F600302088090B6
:1000E60077BAE0FF9077F3E06F60030208809077BD
:1000F600EDE0B44415907724E0B4FF0E63A20190BE
:1001060080A863A2017F06122BC5907B01E06003E5
:100116007401F0907B027464F09077ED7452F09065
:1001260077ECE0646D60030202A37BFF7A14791C0E
:100136001219A77BFF7A1479369077B5E0F52EA3CE
:10014600E0F52FA3E0F530A3E0F531A3E0F532A307
:10015600E0F5331219A7752EFF752F1475309375B8
:1001660031FF75321475339F7BFF7A14796C12193F
:10017600A77BFF7A1479A81219A77BFF7A15790E47
:100186001219A77BFF7A15793B9077BBE0F52EA372
:10019600E0F52FA3E0F530A3E0F5311219A77BFFB8
:1001A6007A1579659077C4E0F52EA3E0F52FA3E0E4
:1001B600F530A3E0F5311219A77BFF7A15799390F4
:1001C60077C8E0F52EA3E0F52FA3E0F530A3E0F520
:1001D600311219A77BFF7A1579C19077B1E0F52E18
:1001E600A3E0F52FA3E0F530A3E0F5311219A77BC4
:1001F600FF7A1579E49077ADE0F52EA3E0F52FA30D
:10020600E0F530A3E0F5311219A77BFF7A167901E4
:100216009077CCE0F52E1219A77BFF7A16792B1270
:1002260019A77BFF7A167954A20EE433F52E12191C
:10023600A77BFF7A167984907AF7E0F52E1219A734
:100246007BFF7A1679AF907B01E0F52E1219A77B1A
:10025600FF7A1679E290772AE0F52E1219A77BFF2E
:100266007A177910A201E433F52E1219A77BFF7ACB
:1002760017793C907AF1E0F52EA3E0F52FA3E0F58F
:1002860030A3E0F531A3E0F532A3E0F5331219A768
:100296001233DB7BFF7A1779871219A7229077EC46
:1002A600E0644C70527E177F8D1236CA9077F4E068
:1002B600F526A3E0F527E4F5287D03AF27AE261241
:1002C60037AB7E177FC81236CAAE26AF27E4FB7D52
:1002D600101238857E177FCB1236CA74102527F583
:1002E60027E43526F5260528E528C3941040CA7E5E
:1002F600177FCB1236CA229077ECE0646C705CF5FF
:100306002A7E177FCD1236CAE4F529AF2A7E007DF4
:10031600031237AB7E177FC81236CAE4F528A82A1F
:10032600E6FF74F62528F582E43477F583EFF005C9
:100336002A0528E528B410E67E777FF6E4FB7D10D3
:100346001238857E177FCB1236CA0529E529C39454
:100356000840B87E177FCB1236CA229077ECE0644D
:100366004B7061F52874DE2528F582E43477F58331
:10037600E0603274DE2528F582E43477F583E0F414
:10038600602374DE2528F582E43477F583E0FF7474
:10039600F42528F582E43477F583E0B507100528BF
:1003A600E528B408C09075787432F0020877907723
:1003B600EC7421F0300A030208777E187F081236A3
:1003C600CA0208779077ECE0B4521A200A077E1822
:1003D6007F101236CA9077EC7472F07E777FEC7DD0
:1003E60008123E2D229077ECE064497045200A07FA
:1003F6007E187F1B1236CA9077F4E0F526A3E0F547
:1004060027E4F528852782852683E0FF74F62528CC
:10041600F582E43477F583EFF00527E527700205CA
:10042600260528E528B480DC7E777FEC7D8A123E9F
:100436002D229077ECE064437079A3E06452704615
:10044600200A077E187F231236CA9077F4E0F52635
:10045600A3E0F527E4F528852782852683E493FF24
:1004660074F62528F582E43477F583EFF00527E561
:1004760027700205260528E528B480DB7E777FEC09
:100486007D8A123E2D229077EDE0645760030208C4
:10049600809077F4E0F526A3E0F52774F62528F595
:1004A60082E43477AD82FC7B80AF27AE26124465AA
:1004B6000208779077ECE06444600302054A90777F
:1004C600F4E0FF64447003020877EFB4310CC20A0B
:1004D6007E187F2C1236CA0208779077F4E0B43083
:1004E6000CD20A7E187F381236CA0208779077F443
:1004F600E0B4320CD20B7E187F451236CA0208775A
:100506009077F4E0B4330CC20B7E187F531236CAD0
:100516000208779077F4E0B4340CD20C7E187F6230
:100526001236CA0208779077F4E0B4350CC20C7E16
:10053600187F6F1236CA0208779077F4E0FF120030
:100546001E020877907578E07013200A077E187FE0
:100556007D1236CA9077EC7421F002087790757890
:100566007432F09077ECE0FFB4510A90800074800A
:10057600F0C2AF80FEEF64577045200A077E187FF1
:100586008B1236CA9077F5E09077A8F0E4F52890BC
:1005960077A8E0FFE528C39F400302087774F62595
:1005A60028F582E43477F583E0FF9077F4E0252898
:1005B6002423F582E43476F583EFF0052880D09085
:1005C60077ECE064536003020679200A077E187F01
:1005D600961236CA9077B5E0FF90762CE06F703CA5
:1005E6009077B6E0FF90762DE06F70309077B7E0A9
:1005F600FF90762EE0B507249077B8E0FF90762F2F
:10060600E0B507189077B9E0FF907630E0B5070CB3
:100616009077BAE0FF907631E06F60169077EC74D1
:1006260021F0300A030208777E187FA51236CA0227
:100636000877E4F528E4F50DAF28FE74232528F5A0
:1006460082E43476F583E0FD1246130528E528C3D7
:1006560094FE40E19080007480F0C2AFE4907FF099
:10066600F0A3F0907FFD74AAF0A374FFF0A3745575
:10067600F080FE9077ECE0644F704C9077F4E0F5F4
:1006860026A3E0F527E5274526700A200A077E18E7
:100696007FAE1236CA200A077E187FB51236CAE424
:1006A600F52874F62528F582E43477F583E0852766
:1006B60082852683F00527E527700205260528E5AD
:1006C60028B480DE0208779077ECE0FFB4452790E7
:1006D60080007480F09077F4E0FDA3E0907FF0CD89
:1006E600F0A3EDF0C2AF907FFD74AAF0A374FFF003
:1006F600A37455F080FEEF64656003020877907777
:10070600F4E0FFA3E0907FF0CFF0A3EFF0E4F5264E
:10071600F527D3907FF1E09527907FF0E09526406E
:1007260020E4F50D2527FFE5263401FE8527828581
:100736002683E0FD1246130527E52770020526806D
:10074600D17E187FB7123D24EF4E60201200039031
:1007560077BBEFF01200039077BCEFF01200039026
:1007660077BDEFF01200039077BEEFF07E187FBDE5
:10077600123D24EF4E60201200039077C4EFF01272
:1007860000039077C5EFF01200039077C6EFF012E2
:1007960000039077C7EFF07E187FC3123D24EF4E1B
:1007A60060201200039077C8EFF01200039077C91B
:1007B600EFF01200039077CAEFF01200039077CBA8
:1007C600EFF07E187FC9123D24EF4E602012000321
:1007D6009077B1EFF01200039077B2EFF0120003BA
:1007E6009077B3EFF01200039077B4EFF07E187FA6
:1007F600CF123D24EF4E60201200039077ADEFF04C
:100806001200039077AEEFF01200039077AFEFF08F
:100816001200039077B0EFF07E187FD5123D24EFDB
:100826004E60081242A49077CCEFF0E4F528E4F588
:100836000DE5282401FFE433FE74AD2528F582E496
:100846003477F583E0FD1246130528E528C3944363
:1008560040DC9080007480F0C2AFE4907FF0F0A39B
:10086600F0907FFD74AAF0A374FFF0A37455F08096
:0A087600FE7E777FEC7D08123E2D18
:010880002255
:10442D00AE07EEC39430400BEED394395005EE2415
:10443D00D0FF22EEC39461400BEED394665005EE8F
:10444D0024A9FF22EEC39441400BEED394465005B0
:08445D00EE24C9FF22AF062284
:1045F900907723E004F07006907722E004F090773A
:0A46090022E0FEA3E0FF1245DD22CF
:100003001245F912442DEFC454F0FEC0061245F90F
:0800130012442DD0E02FFF2262
:1042A400E4907C3FF01245F9907C40EFF0C39430E9
:1042B4004018E0FFD394395011907C3FE0247BF503
:1042C40082E43475F583EFF08011907C3FE0247B29
:1042D400F582E43475F583E4F0800C907C3FE004CF
:1042E400F0E0D3940840BE752E00752F00753000A1
:0C42F400E4F5317B017A75797B122C9C7B
:01430000229A
:043D24008E2B8F2C27
:103D2800907722E4F0A374FFF01245F9EF606EF487
:103D3800606B852C82852B83E493B507EC752D0188
:103D4800E52C252DF582E4352BF583E49360259049
:103D58007723E0252DFF907722E03400FE1245DD21
:103D6800E52C252DF582E4352BF583E493B507047E
:103D7800052D80CCE52C252DF582E4352BF583E443
:103D88009370A6E52D24FFFFE434FFFE907723E02F
:103D98002FF0907722E03EF07E007F0122E4FEFFC4
:013DA80022F8
:1035E4007E197F06123D24EF4E70037F01227E195F
:1035F4007F09123D24EF4E600C1245F9EF24D024CC
:10360400FF920E8002D20E7E197F0F123D24EF4EE0
:10361400600C1245F9EF24D0907AF7F08005E4901D
:103624007AF7F07E197F15123D24EF4E600C124597
:10363400F9EF24D0907B01F08005E4907B01F07ECB
:10364400197F1B123D24EF4E600C1245F9EF24D074
:1036540090772AF08005E490772AF07E197F211272
:103664003D24EF4E600C1245F9EF24D024FF920163
:103674008002C2019077B563A201907AF163A2013E
:103684007F06122BC530013B7E197F27123D24EFA4
:103694004E6030120003907AF1EFF0120003907A3A
:1036A400F2EFF0120003907AF3EFF0120003907A35
:1036B400F4EFF0120003907AF5EFF0120003907A21
:0636C400F6EFF07F00228A
:10271A00C201E4907B01F0D20EC204907AF7F090E5
:10272A00772AF09077B563A201907AF163A2017FCC
:10273A0006122BC5E4F526E52675F003A4242DF52B
:10274A0082E43419F583E493FB740193FA740293D7
:10275A00F912222D700302290CE4F527F528FD74DD
:10276A00A32DF582E43475F583E0FF70030229078F
:10277A00E52675F003A4242DF582E43419F583E4E3
:10278A0093FB740193FA740293F985278275830087
:10279A00122246FEEFB5060875280105270229030D
:1027AA00E5287003022903EE60030228FEE52624C9
:1027BA00FE60281470030228E61470030228EA1443
:1027CA0070030228F21470030228F624056003023B
:1027DA002907907B017401F0022907D20174A32D05
:1027EA00F582E43475F583E0FF642D70030229074E
:1027FA0012442DEFC454F0FC74A42DF582E4347510
:10280A00F583E0FF12442DEF2C907AF1F074A52D98
:10281A00F582E43475F583E0FF12442DEFC454F0D9
:10282A00FC74A62DF582E43475F583E0FF12442D7D
:10283A00EF2C907AF2F074A72DF582E43475F583C3
:10284A00E0FF12442DEFC454F0FC74A82DF582E485
:10285A003475F583E0FF12442DEF2C907AF3F0746F
:10286A00A92DF582E43475F583E0FF12442DEFC4F7
:10287A0054F0FC74AA2DF582E43475F583E0FF1256
:10288A00442DEF2C907AF4F074AB2DF582E4347574
:10289A00F583E0FF12442DEFC454F0FC74AC2DF51F
:1028AA0082E43475F583E0FF12442DEF2C907AF51B
:1028BA00F074AD2DF582E43475F583E0FF12442DF2
:1028CA00EFC454F0FC74AE2DF582E43475F583E060
:1028DA00FF12442DEF2C907AF6F08021D204801D4D
:1028EA00907AF77401F08015C20E801190772A74DD
:1028FA0001F08009E4F528F5270D0227690526026B
:02290A00274163
:01290C0022A8
:10435A009079EDE0C3947C503D9079EDE0FE04F055
:10436A00742B2EF582E43477F583EFF0BF0A279099
:10437A0079EDE0FF04F0742B2FF582E43477F583AE
:10438A00E4F09079EDE0FF123EAF9079ED7408F019
:07439A0090772CE004F022F3
:104301009080007480F09077AD63A201F583F5820F
:1043110063A2017F08122BC59077B563A20190803B
:104321008863A2017F0A122BC5908092E4F0A374E6
:1043310032F0A37401F09077BFE0FF9080B1F0906C
:1043410080E1EFF09080957455F0A3F090800074B7
:0943510001F09080097470F02263
:10402600908009E04410F09080A0E0706C9080A130
:104036007482F09080A874FFF0A3F0A3F0A3F07F41
:10404600039080AEEFF07FCBA3EFF07F039080ACC0
:10405600EFF0A374CBF09080007402F0907C3112E4
:10406600238200000000907C31E0908040F0907C3C
:1040760032E0908041F0907C33E0908042F0907C7A
:1040860034E0908043F0A3E4F0A3F0A3F0A3F09013
:094096008018F0A3F0A3F0A3F0E0
:01409F0022FE
:10417F00908009E04440F09080D17482F09077C035
:10418F00E0FF9080DEF09077C1E0FF9080DFF0904D
:10419F0080027402F0907C351223820000000090A0
:1041AF007C35E0908058F0907C36E0908059F0900C
:1041BF007C37E090805AF0907C38E090805BF0A3E1
:1041CF00E4F0A3F0A3F0A3F0908030F0A3F0A3F0FD
:0241DF00A3F04B
:0141E10022BB
:1040A000908009E04420F09080B8E0706C9080B976
:1040B0007482F07F039080C6EFF07FCDA3EFF07F96
:1040C000039080C4EFF0A374CDF09080C074FFF033
:1040D000A3F0A3F0A3F09080017402F0907C391259
:1040E000238200000000907C35E090804CF0907CB2
:1040F00036E090804DF0907C37E090804EF0907CE0
:1041000038E090804FF0A3E4F0A3F0A3F0A3F09088
:094110008024F0A3F0A3F0A3F059
:014119002283
:103DA9008C268D27A907EAFDE975F018A424ACFF34
:103DB900E5F034808F82F583EDF0EBFDE975F018BD
:103DC900A4FFAEF024ACFBEE34808B82F583A3ED27
:103DD900F08527828C83E0FDEF24A8FFEE3480FE76
:103DE9008F82F583EDF08527828C83A3E08F828E05
:103DF90083A3F0852782852683A3A3E0FDE975F0D7
:103E090018A424A8FFE5F03480FE8F82F583A3A3CC
:103E1900EDF08527828C83A3A3A3E08F828E83A3F1
:043E2900A3A3F0223D
:063E2D008D2BAB07AA0675
:103E3300907C31E0FCA3E0FDA3E0FEA3E0F52F8E30
:103E43002E8D2D8C2CAE02AF038E838F8263A20145
:103E5300E52E540744C0F583852F8263A201AF2B5F
:103E6300122C2E908000E020E5F9E4FCFDFEE52F06
:103E7300252BF52FEE352EF52EED352DF52DEC35C5
:103E83002CF52C908040E52CF0A3E52DF0A3E52E36
:103E9300F0A3E52FF09080007420F0AF2FAE2EAD8D
:0B3EA3002DAC2C907C31122376AF2B4D
:013EAE0022F1
:063FAB008D26AB07AA06FB
:103FB100907C35E0FCA3E0FDA3E0FEA3E0F52A8EB2
:103FC100298D288C27AE02AF038E838F8263A201D5
:103FD100E529540744D0F583852A8263A201AF26DF
:103FE100122C2EE4FCFDFEE52A2526F52AEE3529C4
:103FF100F529ED3528F528EC3527F527908058E58A
:1040010027F0A3E528F0A3E529F0A3E52AF09080A5
:10401100027420F0AF2AAE29AD28AC27907C35126E
:044021002376AF262D
:014025002278
:023A23008F27EB
:103A2500908001E030E5037F0022907C39E0FCA323
:103A3500E0FDA3E0FEA3E0F52B8E2A8D298C2890CE
:103A45007AF163A201E52A540744C8F583852B82E0
:103A550063A2017F06122C44E52B2406F52BE435E1
:103A65002AF52AE43529F529E43528F5289079EF52
:103A750063A201E52A540744C8F583852B8263A216
:103A850001AF27122C44E4FCFDFEE52B2527F52B81
:103A9500EE352AF52AED3529F529EC3528F5289056
:103AA500804CE528F0A3E529F0A3E52AF0A3E52B52
:103AB500F09080017420F0AF2BAE2AAD29AC289090
:073AC5007C39122376AF27C4
:013ACC0022D7
:1034E0009081E0E0F5260526052605260526052619
:1034F00005260526052605260526908010E0F529D7
:10350000A3E0F52AA3E0F52BA3E0F52C9081E1E000
:10351000F526052605260526052605260526052663
:10352000052605260526908014E0F52DA3E0F52E4E
:10353000A3E0F52FA3E0F530E52FB52B08E530B576
:103540002C037F0022E4F526E52F540744E0F583A1
:1035500085308263A2019077EC63A2017F08122C70
:103560005C9077EE63A20190772463A2017F06123C
:103570002BC59077ECE0F527A3E0F528E4F526903D
:1035800077ECE0702AA3E024F8F526E52F540744F1
:10359000E0F58385308274082582F582E43583F571
:1035A0008363A2019077EC63A201AF26122C5CAE7C
:1035B00027E4FCFDE5302528F530E52F3EF52FED1D
:1035C000352EF52EEC352DF52D908014E52DF0A33C
:1035D000E52EF0A3E52FF0A3E530F09080007440D5
:0335E000F0AF2623
:0135E30022C5
:102E40009081E6E0F52605260526052605260526B9
:102E500005260526052605260526908028E0F52965
:102E6000A3E0F52AA3E0F52BA3E0F52C9081E7E0A1
:102E7000F52605260526052605260526052605260A
:102E800005260526052690802CE0F52DA3E0F52EDD
:102E9000A3E0F52FA3E0F530E4F526E52FB52B0AE6
:102EA000E530B52C05C208022F9AE52F540744F0EF
:102EB000F58385308263A2019077EC63A2017F08DD
:102EC000122C5C9077ECE0F527A3E0F528E5284587
:102ED0002770099080027410F07F0022907AF8E049
:102EE000FFF4602D9077EEE06F7076907AF9E0FF56
:102EF0009077EFE06F706A907AFAE0FF9077F0E0F9
:102F00006F705E907AFBE0FF9077F1E06F60228057
:102F1000509077EEE0907AF8F09077EFE0907AF9C1
:102F2000F09077F0E0907AFAF09077F1E0907AFB09
:102F3000F09077ECE0702AA3E024F8F526E52F5412
:102F40000744F0F58385308274082582F582E435E4
:102F500083F58363A2019077EC63A201AF26122C64
:102F60005CAE27E4FCFDE5302528F530E52F3EF585
:102F70002FED352EF52EEC352DF52DAF2CAE2BADDE
:102F80002AAC29AB30AA2FA92EA82DD31223654035
:102F9000099080027410F07F002290802CE52DF0C3
:102FA000A3E52EF0A3E52FF0A3E530F090800274A6
:042FB00040F0AF2618
:012FB40022FA
:10311D009081E3E0F52605260526052605260526DC
:10312D000526052605260526052690801CE0F52991
:10313D00A3E0F52AA3E0F52BA3E0F52C9081E4E0C4
:10314D00F52605260526052605260526052605262A
:10315D00052605260526908020E0F52DA3E0F52E09
:10316D00A3E0F52FA3E0F530E4F526E52FB52B0A06
:10317D00E530B52C05C209023268E52F540744E845
:10318D00F58385308263A20190747863A2017F0E6E
:10319D00122C72907478E0F527A3E0F528907480D6
:1031AD00E0FFF46045907AF1E0FEEF6E706EA3E003
:1031BD00FF907481E06F7064907AF3E0FF907482F9
:1031CD00E06F7058907AF4E0FF907483E06F704C6C
:1031DD00907AF5E0FF907484E06F7040907AF6E09D
:1031ED00FF907485E06F60048032D2D9907478E0DE
:1031FD00702AA3E024F2F526E52F540744E8F58361
:10320D00853082740E2582F582E43583F58363A2C1
:10321D000190747863A201AF26122C72AE27E4FCE4
:10322D00FDE5302528F530E52F3EF52FED352EF552
:10323D002EEC352DF52DAF2CAE2BAD2AAC29AB30A8
:10324D00AA2FA92EA82DD31223655006E5284527B0
:10325D0070099080017410F07F0022908020E52D80
:10326D00F0A3E52EF0A3E52FF0A3E530F09080015B
:05327D007440F0AF26D3
:013282002229
:0436CA008E2B8F2C88
:1036CE00907C31E0FCA3E0FDA3E0FEA3E0F5328E9A
:1036DE00318D308C2FE532FFE5315407FEE42FF5A6
:1036EE002EEE34C0F52D852E82F5837423F0052E33
:1036FE00E52E7002052D532DC7F582852D83740A94
:10370E00F0052EE52E7002052D532DC79077B5636B
:10371E00A201852D83852E8263A2017F06122C2E97
:10372E007406252EF52EE4352DF52D852B83852C4F
:10373E008263A201852D83852E8263A201122C1233
:10374E00908000E020E5F9E4FCFDFE907C31E0F88D
:10375E00A3E0F9A3E0FAA3E02FFFEE3AFEED39FD68
:10376E00EC38FCEF2408FFE43EFEE43DFDE43CFCB7
:10377E00907C31122376907C31E0908040F0907CEA
:10378E0032E0908041F0907C33E0908042F0907C6B
:0C379E0034E0908043F09080007420F034
:0137AA0022FC
:063885008E2B8F2C8D2D0F
:10388B00907C31E0FCA3E0FDA3E0FEA3E0F5338EDA
:10389B00328D318C30E533FFE5325407FEE42FF5E2
:1038AB002FEE34C0F52E852F82F5837423F0052F70
:1038BB00E52F7002052E532EC7F582852E83EBF074
:1038CB00052FE52F7002052E532EC79077B563A2F7
:1038DB0001852E83852F8263A2017F06122C2E7405
:1038EB0006252FF52FE4352EF52E852B83852C827F
:1038FB0063A201852E83852F8263A201AF2D122C2B
:10390B002E908000E020E5F97408252DF52DFFE4BD
:10391B00FCFDFEE5332FF533EE3532F532ED353167
:10392B00F531EC3530F530908040E530F0A3E531E2
:10393B00F0A3E532F0A3E533F09080007420F0AFF4
:0D394B0033AE32AD31AC30907C31122376BA
:01395800224C
:023EAF008F3F43
:103EB100907C31E0FCA3E0FDA3E0FEA3E0F5438E9E
:103EC100428D418C40E543FFE5425407FEE42FFF5C
:103ED100EE34C090772B63A201F5838F8263A20138
:103EE100AF3F122C2E908000E020E5F9E4FCFDFEAE
:103EF100E543253FF543EE3542F542ED3541F541C8
:103F0100EC3540F540908040E540F0A3E541F0A359
:103F1100E542F0A3E543F09080007420F0AF43AE9A
:0B3F210042AD41AC40907C3112237691
:013F2C002272
:0637AB008E2B8F2CAB05F4
:1037B100907C31E0FCA3E0FDA3E0FEA3E0F5328EB6
:1037C100318D308C2FE532FFE5315407FEE42FF5C2
:1037D1002EEE34C0F52D852E82F5837423F0052E4F
:1037E100E52E7002052D532DC7F582852D83EBF053
:1037F100052EE52E7002052D9077B563A201852D6A
:1038010083852E8263A2017F06122C2E7406252E3B
:10381100F52EE4352DF52D532DC7E52B852E82850B
:103821002D83F0052EE52E7002052D532DC7F5824F
:10383100852D83E52CF0052EE52E7002052D532DE7
:10384100C7908000E020E5F9E532240AF532E4353D
:1038510031F531E43530F530E4352FF52F908040E6
:10386100E52FF0A3E530F0A3E531F0A3E532F090C8
:1038710080007420F0AF32AE31AD30AC2F907C318E
:0338810012237699
:013884002221
:1045DD00E5D220E0FBC2AF438E2075D2028F828ED2
:0B45ED0083E0FFE4F5D2538EDFD2AF75
:0145F80022A0
:10461300E5D220E0FBC2AF43D2028F828E83EDF05E
:0946230075D25063D250D2AF22CF
:103F2D00E4FDED2401FFE433FE1245DD74AD2DF506
:103F3D0082E43477F583EFF00DBD3FE6E4FDED242B
:103F4D007FFFE433FE1245DD74A32DF582E4347555
:103F5D00F583EFF074A32DF582E43475F583E070ED
:103F6D001B74A32DF582E43475F5837420F074A4CD
:103F7D002DF582E43475F583E4F080040DBD80BE2B
:103F8D00E4907622F0FDEDFF7E001245DD74232DC9
:0D3F9D00F582E43476F583EFF00DBDFEE90A
:013FAA0022F4
:024465008B2B9F
:10446700A2AF920FC2AF85A22C53A2FE8E838F827A
:1044770005A28C838D827409122C8AE52B53A2FE28
:1044870043A220122C8C53A2DF852CA2A20F92AF3D
:01449700FF25
:014498002201
:1045C000A2AF920FC2AF8C838D82EF122C8A43A2CE
:0C45D00020122C8C53A2DFA20F92AFFF30
:0145DC0022BC
:024578008F268C
:10457A00A2AF920FC2AFE4F5838D827406122C8A21
:10458A00E52643A220122C8C53A2DFA20F92AF7F02
:01459A00011F
:01459B0022FD
:02459C008F2668
:10459E00A2AF920FC2AFE4F5838D82740A122C8AF9
:1045AE00E52643A220122C8C53A2DFA20F92AF7FDE
:0145BE0001FB
:0145BF0022D9
:102AEA00A907E7FFA805EF93C3966008403B74FC6B
:102AFA002FFF80F00F08EF93C3966008402B74FBFA
:102B0A002FFF80E00F08EF93C3966008401B74FA0A
:102B1A002FFF80D00F08EF93D3966008400B74F90B
:102B2A002FFF80C01F1F1F1F1FEF54FEF80303F75C
:102B3A00E893FC08E893FD08E893FE08E893FF226F
:102B4A0009E993C39D6008402974FB29F980F109BA
:102B5A00E993C39E6008401A74FA29F980E209E9E8
:102B6A0093D39F6008400B74F929F980D319191976
:102B7A001919E9C313C313FF22740093F8ECC3981D
:102B8A004024701F740193F8EDC3984019701474AF
:0E2B9A000293F8EEC398400E7009740393F88E
:102BA800EFC39840037F00227F0122EDF8E6F0088A
:102BB800A3DFFA22EDF8E0F608A3DFFA22E0A36328
:102BC800A201F0A363A201DFF475A20022E0A363CF
:102BD800A201F0A363A201E0A363A201F0A363A290
:102BE80001E463A201F0A363A201DFE175A2002260
:102BF800E0A363A2016DFE936CFDEE058393FC15C3
:102C08008363A201DFEA75A200227F00E493A36335
:102C1800A201F00F600CA3E583C2E3F58363A20170
:102C280080EA75A20022E0A363A201F0A3E583C2B3
:102C3800E3F58363A201DFEE75A20022E0A363A29D
:102C480001F0A3E583C2E4D2E3F58363A201DFECDC
:102C580075A20022E583C2E3F583E0A363A201F035
:102C6800A363A201DFEE75A20022E583C2E4D2E3EA
:102C7800F583E0A363A201F0A363A201DFEC75A2D0
:102C88000022F922C002C004C00612FFF0D006D00C
:042C980004D0022240
:103C0A000A536572763A004572724C656E210A0053
:103C1A00205544502054696D654750530A00200AC4
:103C2A00444154414752414D3A20002043414E20DD
:103C3A0054696D654750530A002054726173735377
:103C4A00656E644552520A000ACEF8C4EBE8EDFBF1
:103C5A0043414E210A000A45727241647243414E41
:103C6A003A000A00205265496E69742043414E0A9F
:103C7A00002043414E283029203E20544F210A007B
:0E3C8A0020545520300A0020545520310A00E5
:03001E00E4FF22DA
:10452900C2A9438902758C48758A4875D90475DB17
:104539004875DC4875DD4875DE48E4F5E9F5F9D2DA
:08454900D9C2DAD28CD2DE22C5
:1044FB00C2D9907B17E07013E5E92419F5EB30D79F
:10450B0006E5F904F5FB2285F9FB22E5E924C8F55C
:0E451B00EB30D706E5F904F5FB2285F9FB220B
:1043A100C2D9907B17E0702C301C16E5E92432F558
:1043B100EB30D707E5F904F5FB800385F9FBC21C57
:1043C10022E5E92405F5EB30D706E5F904F5FB22F2
:1043D10085F9FB22E5E92432F5EB30D706E5F9044E
:0743E100F5FB2285F9FB2228
:10455100124529907B17E0C39464500612411A1248
:1045610044FB120022D21BE4F555907C2FF0F54458
:07457100F559C21CF55722A9
:1043E800EF24FCF544200A127E3C7F0A1236CA7E6E
:1043F800777FF0E4FBAD44123885E544D3940D4053
:1044080010200A077E3C7F111236CAE4F544D219FF
:10441800229077F063A201907C1F63A201AF44123F
:054428002BC5C21922A2
:0F464000D3EF6480948D5006E55970028F592294
:101F680020D903022045201B03022045E559605271
:101F7800907478540FFF7D46122BBCE546640170BF
:101F88001E907480E0B4FF0ED21D200A127E3C7FA2
:101F98001A1236CA8009301D06E4F5590220451286
:101FA80044FB1241E2200A077E3C7F281236CA20F1
:101FB8000A0B7E747F78E4FBAD59123885E4F55935
:101FC800807BE5446043907C23E02405F526D39488
:101FD8000D4007E4F544D2198063907C1FE5265430
:101FE8000FFF7D46122BBCE54630E702D21CE546C2
:101FF800B40109301D06E549640160031241E2128B
:1020080044FBE4F544D2198034E556601E907B0306
:10201800540FFF7D46122BBCE546B40103201D0377
:102028001241E21244FBE4F5568012201E0C907B0C
:1020380017E0C3946450031242441244FB123283E3
:102048008F26EF700302210C1243A1E4F557E546F1
:10205800B4010CD21D200A077E3C7F351236CAE532
:1020680058C394C8502D30032AE546B4420DE549BB
:10207800B4020890772AE06401601874182558F5AE
:1020880082E4347BF583E5262558F5587D46AF264E
:10209800122BB3300121E54620E71C9079EF7D46ED
:1020A800AF26122BB3AF26123A23EF700A200A0785
:1020B8007E3C7F431236CAE54654817047E526D3F5
:1020C800940D400C200A3D7E3C7F521236CA803463
:1020D800E548D394074028200A2A7E3C7F601236C0
:1020E800CA90757B7D46AF26122BB37E757F7BE445
:1020F800FBAD261238857E3C7F6C1236CA8005AF50
:1021080026123959300D2030001B907B17E0C394FC
:102118006450120557E55794F0400A908000748087
:10212800F0C2AF80FEC20D200203022227E55560EF
:1021380031D39401400415558028907C2FE004F099
:10214800E0D39403400D200A077E3C7F6E1236CA06
:10215800124551200A077E3C7F7B1236CAE4F555AA
:10216800D21B301A43E556703F907B0304F0A374EA
:1021780008F0A37480F0A37401F0A37406F0907CB7
:102188001AE0907B08F0907C1BE0907B09F0907C33
:102198001CE0907B0AF0907C1DE0907B0BF0E4A3A0
:1021A800F0A3F075560BC21A301872907C18E070C4
:1021B80035E5567031907B037442F0A37408F090B3
:1021C8007C19E0907B05F0907C1EE0907B06F0A3E4
:1021D8007401F0755606200A077E3C7F8A1236CABB
:1021E800907C18E004F0907C18E06402702FE556AB
:1021F800702B907B037402F0A37408F0907C19E0B4
:10220800907B05F0A3F0A37401F0755606200A0729
:102218007E3C7F911236CA907C18E004F0C202120C
:0422280024C0C2000C
:01222C00228F
:10449900E558602CE49078ECF0A3E558F0907AF0B8
:1044A900E09078EEF0A37419F0907B1863A2019064
:1044B90078F063A201AF58122BC5E4F5587F0122A9
:0344C9007F00224F
:0B464F00301905C2197F01227F0022F4
:0100210022BC
:06467400E4F558F54422B4
:0A465A00E490757BF0A3F0A3F022BA
:1044CC002043616E457247495400200A00457272C0
:1044DC004C656E43616E21000A002043616E45728B
:0F44EC0072434821000A20526571457272210007
:10328300E59B541F6020200A1A7E447FCC1236CA65
:10329300E59B541FFF7E007D031237AB7E447FD630
:1032A3001236CAE4F59BE5BA30E010E4F5B375B124
:1032B30080F5B2D21BF555907C2FF0E5CFF4700367
:1032C3000233D8752801E4F527E5CFF455287003B8
:1032D3000233C6E527C454F0F5B1E5B2547F642048
:1032E3006003023397E5B3540FF54A85BC46E5BD49
:1032F300541FFF131313541FFFE5BD54E044184F2D
:10330300F547E5BDC43354E0FFE5BE131313541F63
:103313004FF548E5BEC43354E0FFE5BF1313135420
:103323001F4FF54985A34B85A34C85A34D85A34E1C
:1033330085A34F85A35085A35185A352E4F5B220FD
:103343001E0CE546547EB5460575B350800375B330
:10335300D0E54A700AE546547EB546037F00223025
:103363001E08E54630E7037F0022E54AD394084070
:103373001D200A177E447FD91236CAAF4A7E007DCC
:10338300031237AB7E447FE41236CA7F0022E54A3C
:103393002405FF22E5B2549F6023200A207E447F48
:1033A300E61236CAAFB27E007D031237ABAFB37EEF
:1033B300007D031237AB7E447FE41236CAE4F5B2D4
:1033C30075B3D0E52825E0F5280527E527C394083C
:0733D30050030232CC7F0021
:0133DA0022D0
:1041E200907B17E0C39464505675B180E4F5B3F543
:1041F200B28546BCE548C4135407FFE54754E04F77
:10420200F5BDE54833333354F8FFE549C413540789
:104212004FF5BEE54933333354F8F5BF854BA385DB
:104222004CA3854DA3854EA3854FA38550A38551ED
:10423200A38552A3E54A540F2450F5B375550AC21B
:024242001B223D
:1042440075B190E5B220E613200A107E447FF11286
:1042540036CAAFB27E007D031237ABE4F5B3F5B2D4
:104264007471250FF582E43461F583E0F5BCE4F55F
:10427400BD7472250FF582E43461F583E0FF3333B6
:104284003354F8F5BE75BF78050F050F7471250F0B
:10429400F582E43461F583E07002F50F75B35022C2
:09466400EF6003C29622D29622F7
:10411A0043AB01C2E8C2EAE4FFEFC454F0F5B1C30D
:10412A00EF64809488500575B3D08003E4F5B3E456
:10413A00F5B2F5BCF5BDF5BEF5BFF5C4F5C5F5C6D6
:10414A00F5C7F5A3F5A3F5A3F5A3F5A3F5A3F5A381
:10415A00F5A30FBF0EC3907B17E0FF25E0F5B475FA
:10416A00B50C75B66C75A11275AB0275C13E75C3F7
:04417A00FF75C20308
:01417E00221E
:100EA2003E2A2C312CCFE0F0E0ECE5F2F0FB20F30F
:100EB200EFF0E0E2EBFFFEF9E5E3EE20EAEEEDF221
:100EC200F0EEEBEBE5F0E020CACF20C8F1E5F2FC52
:100ED2000A003E4C2C6B30312C25732C43EAEEF089
:100EE200EEF1F2FC20EDE020F8E8EDE52043414E82
:100EF2002C30202D20353030EAE1283530EC292CF9
:100F020031202D203530EAE128353030EC290A0035
:100F120030202D20353030EAE1283530EC290031FF
:100F2200202D203530EAE128353030EC29003E53BF
:100F32002C6B30322C2562752CCCE0EAF12E20E0AD
:100F4200E4F0E5F120E1EBEEEAE020D2D128302D09
:100F520038290A003E532C6B30332C2562752CCC79
:100F6200E0EAF12E20E0E4F0E5F120E1EBEEEAE048
:100F720020D2C8D228302D38290A003E532C6B309B
:100F8200342C2562752CCCE0EAF12E20E0E4F0E569
:100F9200F120E1EBEEEAE020D2D328302D38290A05
:100FA200003E422C6330312C2562752CC2F2EEF0E9
:100FB200E8F7EDFBE920EAEEEDF2F0EEEBEBE5F01F
:100FC20020EDE020F8E8EDE50A003E2A2C312CCF96
:100FD200F0EEF2EEEAEEEB20C8F1E5F2FC2DCCE009
:100FE200E3E8F1F2F0E0EBFCEDFBE920EDE020EFCD
:100FF200EEF0F2F32052533233320A003E4C2C6BA5
:1010020030352C256C752CD1EAEEF0EEF1F2FC2095
:10101200EEE1ECE5EDE020EDE020EFEEF0F2F32C76
:101022003130302C3230302C3330302C3630302CC2
:10103200313230302C323430302C343830302C399C
:101042003630302C31393230302C33383430302C89
:1010520035373630302C3131353230300A003E539C
:101062002C6B30362C2562752CC0E4F0E5F120CAD9
:10107200CF20E4EBFF20ECE0E3E8F1F2F0E0EBE874
:101082000A003E532C6B31312C2562752CC0E4F0E2
:10109200E5F120F0E5F2F0E0EDF1EBFFF2EEF0E049
:1010A2000A003E532C6B31322C2562752CCAEEEBB2
:1010B2002DE2EE20E1EBEEEAEEE220E220EEF2E2B9
:1010C200E5F2E52028EFE0EAE5F23D352B6E2A3124
:1010D2003320E1E0E9F2290A003E532C6B31332C34
:1010E2002562752CC7E0E4E5F0E6EAE020F1F2E0E3
:1010F200F0F2E020EFE5F0E5E4E0F7E828ECF12992
:101102000A003E422C6B30392C2562752CCDE5202D
:10111200EFE5F0E5E4E0E2E0F2FC20E4E8E0E3ED14
:10112200EEF1F2E8EAF30A003E422C6B31302C2554
:1011320062752CCFE5F0E5E7E0E3F0F3E7EAE020C3
:10114200EFF0E820EEF2F1F3F2F1F2E2E8E820EE5D
:10115200E1ECE5EDE0203220ECE8ED2E0A003C2146
:10116200003C6B30313D003C6B30323D003C6B301B
:10117200333D003C6B30343D003C6330313D003C3C
:101182006B30353D003C6B30363D003C6B31313DC0
:10119200003C6B31323D003C6B31333D003C6B30E7
:1011A200393D003C6B31303D00CEF820E4EBE8EDF8
:1011B200FB210A000A4173796E634F55543A000AC3
:1011C200435243204552523A20000A4173796E63DA
:1011D200494E3A00CFE0EAE5F220E22043414E0ACE
:1011E20000D2D320320A00D2D320330A00C0F0F555
:1011F200D2D10A003F3F3F0A000089129B24AD363C
:10120200BF48C15AD36CE57EF78108931AA52CB763
:101212003EC940DB52ED64FF76028B109926AF3453
:10122200BD4AC358D16EE77CF5830A9118A72EB543
:101232003CCB42D950EF66FD74048D169F20A93233
:10124200BB4CC55ED768E17AF3850C971EA128B323
:101252003ACD44DF56E960FB72068F149D22AB3013
:10126200B94EC75CD56AE378F1870E951CA32AB103
:1012720038CF46DD54EB62F97008811A932CA53EF3
:10128200B740C952DB64ED76FF89009B12AD24BFE3
:1012920036C148D35AE56CF77E0A8318912EA73CD3
:1012A200B542CB50D966EF74FD8B029910AF26BDC3
:1012B20034C34AD158E76EF57C0C851E9728A13AB3
:1012C200B344CD56DF60E972FB8D049F16A920BBA3
:1012D20032C54CD75EE168F37A0E871C952AA33893
:1012E200B146CF54DD62EB70F98F069D14AB22B983
:1012F20030C74ED55CE36AF1780011233246576558
:10130200748C9DAFBECADBE9F810013322564775D3
:10131200649C8DBFAEDACBF9E821300213677644C4
:1013220055ADBC8E9FEBFAC8D931201203776654B3
:1013320045BDAC9E8FFBEAD8C942536170041527A4
:1013420036CEDFEDFC8899ABBA5243716014053793
:1013520026DECFFDEC9889BBAA6372405125340684
:1013620017EFFECCDDA9B88A9B7362504135241673
:1013720007FFEEDCCDB9A89A8B8495A7B6C2D3E15C
:10138200F008192B3A4E5F6D7C9485B7A6D2C3F153
:10139200E018093B2A5E4F7D6CA5B48697E3F2C044
:1013A200D129380A1B6F7E4C5DB5A49687F3E2D033
:1013B200C139281A0B7F6E5C4DC6D7E5F48091A324
:1013C200B24A5B69780C1D2F3ED6C7F5E49081B313
:1013D200A25A4B79681C0D3F2EE7F6C4D5A1B08204
:1013E200936B7A48592D3C0E1FF7E6D4C5B1A092F3
:0913F200837B6A58493D2C1E0F53
:03002300023ACDD1
:0D3ACD00C0E0C0F0C083C082C0D075D0182A
:103ADA0030985AC298750B01AF99201F13BF550928
:103AEA00756100D21FD2918044906F30EFF0803D13
:103AFA00E56B703474322561F582E4346FF583EF37
:103B0A00F0E561B40104EF04F55DE561600AB55DB5
:103B1A001304F56BC291800CEF64556007C21F90C5
:103B2A006F30EFF005618005906F30EFF030992922
:103B3A00302024D290E568B5600DC220D222C2900E
:103B4A00E4FF124664801074322568F582E434700A
:093B5A00F583E0F5990568C299B4
:0B3B6300D0D0D082D083D0F0D0E03270
:1033DB007BFF7A0E79A21219A7907B17E0701475F8
:1033EB002EFF752F0F7530127BFF7A0E79D41219C1
:1033FB00A78012752EFF752F0F7530217BFF7A0E6C
:10340B0079D41219A77BFF7A0F7930906170E0F5B0
:10341B002E1219A77BFF7A0F795690616BE0F52E70
:10342B001219A77BFF7A0F797D906102E0F52E12BE
:10343B0019A77BFF7A0F79A3A21EE433F52E12197D
:10344B00A77BFF7A0F79CC1219A7907472E0FEA3B9
:10345B00E0FFC3E49FFFE49EFEAB07FA3395E0F970
:10346B00F87F007E8C7D0A7C001222C58F318E3056
:10347B008D2F8C2E7BFF7A0F79FE1219A77BFF7A8B
:10348B00107960856A2E1219A77BFF7A10798490C8
:10349B006845E0F52E1219A77BFF7A1079A4906F7F
:1034AB002EE0F52E1219A77BFF7A1079DB90616E57
:1034BB00E0F52E1219A77BFF7A117904A221E433D0
:1034CB00F52E1219A77BFF7A11792A906F31E0F54F
:0534DB002E1219A722CA
:102FB5007E117F60123D24EF4E70037F0122E49065
:102FC5007B17F07E117F63123D24EF4E601512458D
:102FD500F9BF3106907B17740AF0BF3206907B1754
:102FE5007464F09061027402F090616BF09061700E
:102FF500F07E117F69123D24EF4E60081242A490C5
:103005006170EFF07E117F6F123D24EF4E60081264
:1030150042A490616BEFF07E117F75123D24EF4E57
:1030250060081242A4906102EFF07E117F7B123D91
:1030350024EF4E600D1242A4EC4D4E4F24FF921E1C
:103045008002C21E7E117F81123D24EF4E60231245
:1030550042A4A804A905AA06AB077F007E8C7D0AB9
:103065007C001222C5122357907472EEF0A3EFF084
:10307500800A90747274FFF0A374B8F07E117F8794
:10308500123D24EF4E60071242A48F6A8003756AD1
:10309500017E117F8D123D24EF4E600A1242A490ED
:1030A5006845EFF08005E4906845F07E117F931246
:1030B5003D24EF4E600A1242A4906F2EEFF0800679
:1030C500906F2E7401F07E117F99123D24EF4E60B2
:1030D5000A1242A490616EEFF08005E490616EF0F3
:1030E5007E117F9F123D24EF4E600C1245F9EF24AF
:1030F500D024FF92218002D2217E117FA5123D248A
:10310500EF4E600C1245F9EF24D0906F31F0800539
:07311500E4906F31F07F0030
:01311C002290
:10290D00C220C222C21FE4906F2FF0F568F560F56A
:10291D00089061A4F0F561F50B90747274FFF0A34B
:10292D0074F4F0122FB5E4F50F907C3D7461F0A3B3
:10293D007471F0906170E0F50FE50FC394014007DD
:10294D00E50FD394084003E4F50FE50F6028907C64
:10295D003DE475F00112227385F082F58374C4F0A5
:10296D00150F907C3DE475F00112227385F082F510
:10297D0083E50FF080D490616BE0F50FE50FC39404
:10298D00014007E50FD394084003E4F50FE50F6010
:10299D0028907C3DE475F00112227385F082F58359
:1029AD0074C8F0150F907C3DE475F001122273850B
:1029BD00F082F583E50FF080D4906102E0F50FE52C
:1029CD000FC394014007E50FD394084003E4F50FBE
:1029DD00E50F6028907C3DE475F00112227385F0BF
:1029ED0082F58374C2F0150F907C3DE475F00112F1
:1029FD00227385F082F583E50FF080D4907C3DE461
:102A0D0075F00112227385F082F583E4F0907C3D20
:102A1D0075F00112227385F082F583E4F0F50FF560
:102A2D0069E4F55B75F075E569A42453F582E5F06D
:102A3D003468F58375F00DE55B1223B3E4F0055BA7
:102A4D00E55BB408DF75F075E569A42446F582E50C
:102A5D00F03468F583E4F0E56975F00DA42403F511
:102A6D0082E43461F583E4F0F55F75F068E569A4FF
:102A7D002432F582E5F03471F58375F00DE55F12C2
:102A8D0023B3E4F0055FE55FB408DF0569E569642C
:102A9D0008708EE4F56FF55AF55CF55EF567F56C2B
:102AAD00F55FF55BF569F566C2ADF5C9D2CDD2CC52
:102ABD00C2C9C2CAF5CDF5CC907472E0F5CBA3E0D6
:102ACD00F5CA85CBCD85CACCD29ED29CD2CAC2AC1A
:0C2ADD00C298C29975B81075B710D2AC41
:012AE90022CA
:0100220022BB
:103959008F2730210EE546B44209E5496402700318
:10396900023A22E54754E324DF604A24DF60291440
:10397900602624E3605C24E0601E24606003023A50
:1039890022E54875F00DA42403F582E43461F5833A
:103999007D46AF27122BB32275F00DE55EA424EE08
:1039A900F582E5F0346BF5837D46AF27122BB3051D
:1039B9005E535E3F2275F00DE55AA424C5F582E5F4
:1039C900F03461F5837D46AF27122BB3055A535A5C
:1039D9007F2275F075E548A42453F582E5F0346833
:1039E900F583E549543FFF1313543F75F00D122336
:1039F900B37D46AF27122BB375F068E548A424328E
:103A0900F582E5F03471F583E549543FFF1313540A
:0A3A19003F75F00D1223B3E4F02214
:101CA100E4F528906F2EE0FFE528C39F4003021E54
:101CB100B9E55E655C605A75F00DE55CA424F2F54A
:101CC10082E5F0346BF583E02405F529C3940E50C9
:101CD1002E75F00DE55CA424EEF582E5F0346BF58C
:101CE1008363A20174022566F582E43460F583639F
:101CF100A201AF29122BC5E5292566F566800A20C8
:101D01000A077E117FAB1236CA055C535C3F021E87
:101D1100B475F075E569A42453F582E5F03468F5EE
:101D21008375F00DE55B1223B3E07003021DD575D9
:101D3100F075E569A42457F582E5F03468F58375FB
:101D4100F00DE55B1223B3E02405F529C3940E5091
:101D51003675F075E569A42453F582E5F03468F52C
:101D61008375F00DE55B1223B363A201740225664E
:101D7100F582E43460F58363A201AF29122BC5E536
:101D8100292566F566800A200A077E117FAB123687
:101D9100CA75F075E569A42453F582E5F03468F558
:101DA1008375F00DE55B1223B3E4F0055BE55BC3DE
:101DB10094085003021EB4E4F55B75F075E569A45F
:101DC1002446F582E5F03468F583E4F0056953694A
:101DD10007021EB4E55A656F605A75F00DE56FA4F0
:101DE10024C9F582E5F03461F583E02405F529C3C2
:101DF100940E502E75F00DE56FA424C5F582E5F023
:101E01003461F58363A20174022566F582E43460CE
:101E1100F58363A201AF29122BC5E5292566F56675
:101E2100800A200A077E117FAB1236CA056F536FF5
:101E31007F021EB4E56775F00DA42403F582E43436
:101E410061F583E06068E56775F00DA42407F5820C
:101E5100E43461F583E02405F529C3940E502DE5A2
:101E61006775F00DA42403F582E43461F58363A260
:101E71000174022566F582E43460F58363A201AF43
:101E810029122BC5E5292566F566800A200A077EF9
:101E9100117FAB1236CAE56775F00DA42403F582F4
:101EA100E43461F583E4F00567536707800505674E
:101EB1005367070528021CA4856629E4F56690701E
:101EC100327455F0A3F0E5292405A3F0E4A3F0A3AF
:101ED100E56AF0906845E0907037F0E5296011906F
:101EE100600263A20190703863A201AF29122BC571
:101EF100E4F562F563E5292403F56590703563A285
:101F0100019011FB63A201AF65AE64AD63AC6212D7
:101F11002BF88F658E648D638C6274382529F58268
:101F2100E43470F583E563F074392529F582E434EE
:101F310070F583E562F0E5292408F560D220E4F527
:101F41006890616FF07F01124664C2992099FDD2B9
:101F510099200A127E117FB61236CA7E707F32E452
:061F6100FBAD60123885A3
:011F67002257
:1024C000E56775F00DA42403F582E43461F583E03B
:1024D0007005056753670775F075E569A42453F522
:1024E00082E5F03468F58375F00DE55B1223B3E007
:1024F0007023055BE55BC39408401AE4F55B75F057
:1025000075E569A42446F582E5F03468F583E4F0C6
:102510000569536907300020C200906F31E06012F6
:1025200004F0E0D394F0400A9080007480F0C2AFD1
:1025300080FE90616FE004F030DA3FC2DA9061A46F
:10254000E0FF906F2FE0FDC39F502FE56E25ECF567
:10255000EC30D709E56D25FC04F5FC8006E56D251A
:10256000FCF5FC74A52DF582E43461F583E0B56AD1
:1025700003121CA1906F2FE004F030200F90616FC8
:10258000E0D39414400BC220D2228005E490616F06
:10259000F0906F30E0FF600C7E007D031237ABE4FB
:1025A000906F30F0E56B7003022719F527E4F562B0
:1025B000F563E52724FEF565906F3463A201901161
:1025C000FB63A201AF65AE64AD63AC62122BF88F02
:1025D000658E648D638C62C21FE4F56BE5634562B2
:1025E0006022300A030227197E117FC11236CA7E8B
:1025F0006F7F32E4FBAD271238857D03AF63AE6297
:102600001237AB22200A127E117FCC1236CA7E6F9F
:102610007F32E4FBAD27123885906F34E0FB640114
:1026200060030226B4906F36E09061A3F06007E08B
:1026300020E7030227199061A3E0547FF0906845DA
:10264000F0E5E92402F5EC30D707E5F904F5FC8064
:102650000385F9FCC2DA906F35E075F064A485F06B
:102660006DF56E906F37E0FE541F9061A4F0EE544C
:10267000E0600E906F37E0FFC413540704906F2E94
:10268000F0E4906F2FF0F5279061A4E0FFE527C3F9
:102690009F400302271974382527F582E4346FF52B
:1026A00083E0FF74A52527F582E43461F583EFF01C
:1026B000052780D4906F35E0656A705DEB24FD607E
:1026C0002D14603514603D24037044200A077E11E8
:1026D0007FD61236CAE556704075560D906F376337
:1026E000A201907B0363A201AF56122BC522200AE0
:1026F000287E117FE31236CA22200A1D7E117FE94F
:102700001236CA22200A127E117FEF1236CA222008
:092710000A077E117FF61236CA99
:01271900229D
:103CA400020881E493A3F8E493A34003F68001F2AD
:103CB40008DFF48029E493A3F85407240CC8C33321
:103CC400C4540F4420C8834004F456800146F6DFF0
:103CD400E4800B010204081020408090466DE47ECD
:103CE400019360BCA3FF543F30E509541FFEE493E5
:103CF400A360010ECF54C025E060A840B8E493A3AC
:103D0400FAE493A3F8E493A3C8C582C8CAC583CAD6
:103D1400F0A3C8C582C8CAC583CADFE9DEE780BE8E
:014673000046
:10222D00BB010689828A83E0225002E722BBFE02AF
:09223D00E32289828A83E49322E2
:10224600BB010CE58229F582E5833AF583E022504D
:1022560006E92582F8E622BBFE06E92582F8E22297
:0D226600E58229F582E5833AF583E49322B1
:10227300A3F8E0C5F025F0F0E5821582700215831E
:06228300E0C838F0E8227B
:1022890075F008758200EF2FFFEE33FECD33CDCC0C
:1022990033CCC58233C5829BED9AEC99E58298408F
:1022A9000CF582EE9BFEED9AFDEC99FC0FD5F0D66C
:1022B900E4CEFBE4CDFAE4CCF9A88222B800C1B996
:1022C9000059BA002DEC8BF084CFCECDFCE5F0CBD4
:1022D900F97818EF2FFFEE33FEED33FDEC33FCEB0D
:1022E90033FB10D703994004EB99FB0FD8E5E4F9C8
:1022F900FA227818EF2FFFEE33FEED33FDEC33FCB5
:10230900C933C910D7059BE99A4007EC9BFCE99AA8
:10231900F90FD8E0E4C9FAE4CCFB2275F010EF2FED
:10232900FFEE33FEED33FDCC33CCC833C810D707ED
:102339009BEC9AE899400AED9BFDEC9AFCE899F828
:0E2349000FD5F0DAE4CDFBE4CCFAE4C8F922BB
:0E235700C3E49FFFE49EFEE49DFDE49CFC2297
:10236500EB9FF5F0EA9E42F0E99D42F0E89C45F0CE
:012375002245
:0C237600ECF0A3EDF0A3EEF0A3EFF022DA
:10238200A8828583F0D083D08212239912239912D6
:102392002399122399E473E493A3C583C5F0C583FB
:1023A200C8C582C8F0A3C583C5F0C583C8C582C8A5
:0123B2002208
:0C23B300A42582F582E5F03583F5832235
:10194500E53A242EF8E6053A22782B301602782E51
:10195500E475F00112242002222D200FEB7F2ED2F8
:101965000F8018EF540F2490D43440D4FF30130B5C
:10197500EF24BFB41A0050032461FFE53B60021554
:101985003B053EE53E7002053D30160D782BE475AE
:10199500F001122420EF0223BF02435A7403D2162A
:1019A5008003E4C216F53A8B2B8A2C892DE4F53B8E
:1019B500F53DF53EE53B60077F2012198080F57502
:1019C5003CFFC210C20FC211C212C214C215C21707
:1019D50012194EFF700D3016057F00121991AF3E9A
:1019E500AE3D22B4255FC2D5C21312194EFF24D0D5
:1019F500B40A00501A75F00A783B30D50508B6FFD1
:101A05000106C6A426F620D5047002D21280D92478
:101A1500CFB41A00EF5004C2E5D213021B91D210C5
:101A250080C6D20F80C0D21180BCD2D580BAD21464
:101A350080B47F201219802011077401B53B004046
:101A4500F1121945FF1219800219B9D217D2158062
:101A550095121945FB121945FA121945F94A4B70A9
:101A65000679627A1C7BFF20112EE53B602A7E00F9
:101A75008E8275830012224660060EEE653C70F07C
:101A8500C2D5EBC0E0EAC0E0E9C0E0EE121BD8D059
:101A9500E0F9D0E0FAD0E0FB12222DFF60AAEBC0FE
:101AA500E0EAC0E0E9C0E0121980D0E02401F9D0F5
:101AB500E03400FAD0E0FBE53C0460DCD53CD9809D
:101AC500877BFF7A1B79D4D211809C7910800279AB
:101AD50008C215C2178008D2D5790A8004790AC2CE
:101AE500D5E53C047002F53CE4FAFDFEFF1219450C
:101AF500FC7B08201013121945FD7B10300F0A12CC
:101B05001945FE121945FF7B20EC3382D592D5503D
:101B150013C3E4300F069FFFE49EFEE42010039DEF
:101B2500FDE49CFCE4CBF8C210EC700CCFCECDCC20
:101B3500E824F8F870F38017C3EF33FFEE33FEEDBA
:101B450033FDEC33FCEB33FB994002FB0FD8E9EB9B
:101B5500301005F8D0E0C448B210C0E00AEC4D4E94
:101B65004F78207B0070C2EAB53C0040BCC0E01253
:101B75001BDAD0F0D0E0201004C4C0E0C4B210C01D
:101B8500F0121969D0F0D5F0EB0219B912247F1AB9
:101B950056531AD0581A274C1A23421AD44F1ADC16
:0F1BA500441ADC491A3C431AE2551AC6461AC6BE
:101BB400451AC6471C82501A2B2D1A2F2E1A522B47
:101BC4001A33231A50201C6B2A19EB4800001A4AB6
:101BD4003F3F3F00790AA2D5201214301409B910EE
:101BE400020404B9080104A2D520150250010420FE
:101BF40011689211B53B005034C0E07F20301219B7
:101C04007F30A21172157214500F121C31C211C20E
:101C140015C214C2177F30800F301403E9C0E012DC
:101C24001980301403D0E0F9D0E0B53BCC30141760
:101C34007F30B9100C1219807F583013077F7880D9
:101C440003B908031219803011057F2D0219807F12
:101C5400202017F87F2B2015F322921180CF286EB5
:101C6400756C6C2900D2101219453010F8C2107826
:101C74003B30D50108F60219EB2D5043495812198F
:101C8400452403B405004001E4901C7D93121971AE
:0D1C9400743A121971D212753B04021AD075
:102C9C008B2B8A2C892DE4F537F536F535F534F583
:102CAC0032F533E52F4530452E6012EBC0E0EAC01B
:102CBC00E0E9C0E0AB2EAA2FA930122430AB2B05D3
:102CCC002DE52DAA2C7002052C14F912222DF538A5
:102CDC00C394094007E538D3940D40E1E5386420EE
:102CEC0060DBE538B42D054333038016E538B42B8F
:102CFC0005433301800C74FF252DF52D74FF352C05
:102D0C00F52CE53160046410703FAB2BAA2CA92D77
:102D1C0012222D64306009E531702E75310A80293C
:102D2C00900001122246FF64786004EFB4581343FC
:102D3C0033017531107402252DF52DE4352CF52C4D
:102D4C008007E5317003753108AB2B052DE52DAAF5
:102D5C002C7002052C14F912222DF538C394614005
:102D6C000AE538D3947A50035338DF74D02538F5FC
:102D7C0038C3940A400CE5389411406D74F9253829
:102D8C00F538E538D39531506043330185373C85B0
:102D9C00363B85353A853439AF317E00E4FCFDABEA
:102DAC0037AA36A935A8341223D1C8ECC8C9EDC945
:102DBC00CAEECACBEFCBE4FCFDFEEB2538F537EEC3
:102DCC003AF536ED39F535EC38F534AF37AE36AD7E
:102DDC0035FCAB3CAA3BA93AA839D3122365500366
:102DEC00022D55433304022D55E53320E003E480D6
:102DFC002DE52F4530452E601EAB2BE52D24FFF91C
:102E0C00E52C34FFFAEBC0E0EAC0E0E9C0E0AB2E01
:102E1C00AA2FA930122430E53330E20774FFFFFEED
:102E2C00FDFC22E533AF37AE36AD35AC3430E103C3
:042E3C0002235722F4
:1023BF00BB010689828A83F0225002F722BBFE01FD
:0223CF00F322F7
:1023D100E88FF0A4CC8BF0A42CFCE98EF0A42CFCAB
:1023E1008AF0EDA42CFCEA8EF0A4CDA8F08BF0A429
:1023F1002DCC3825F0FDE98FF0A42CCD35F0FCEB88
:102401008EF0A4FEA9F0EB8FF0A4CFC5F02ECD394C
:0F241100FEE43CFCEAA42DCE35F0FDE43CFC22B9
:10242000FAE6FB0808E6F925F0F618E6CA3AF622BD
:10243000BB011A89828A83D0F0D0E0F8D0E0F9D0CD
:10244000E0FAD0E0FBE8C0E0C0F00224AE5016E9AC
:10245000F8D083D082D0E0F9D0E0FAD0E0FBC0829F
:10246000C0830224A5BBFE16E9F8D083D082D0E059
:0F247000F9D0E0FAD0E0FBC082C0830224B7228B
:10247F00D083D082F8E4937012740193700DA3A3EC
:10248F0093F8740193F5828883E473740293686000
:06249F00EFA3A3A380DF00
:0924A500EBF608EAF608E9F6225C
:0924AE00EBF0A3EAF0A3E9F0222F
:0924B700EBF208EAF208E9F22256
:00000001FF
